:0200000480007A
:100000006F000005732F2034930F80006308FF03F7
:10001000930F90006304FF03930FB0006300FF038E
:10002000130F000063040F0067000F00732F2034CC
:1000300063540F006F00400093E19153171F0000BD
:1000400023223FFC171F000023200FFC6FF01FFF2F
:100050009300000013010000930100001302000050
:100060009302000013030000930300001304000038
:100070009304000013050000930500001306000020
:100080009306000013070000930700001308000008
:10009000930800001309000093090000130A0000F0
:1000A000930A0000130B0000930B0000130C0000D8
:1000B000930C0000130D0000930D0000130E0000C0
:1000C000930E0000130F0000930F0000732540F102
:1000D0006310050097020000938202017390523072
:1000E000735044749702000093820201739052305F
:1000F00073500018970200009382020273905230EE
:10010000B70200809382F2FF7390023B9302F001EA
:100110007390023A7350403097020000938242017C
:100120007390523073502030735030309301000080
:1001300097020000938242ED739052301305100035
:100140001315F501634C05000F00F00F930110002B
:100150009308D0051305000073000000930200000F
:10016000638A020073905210B7B20000938292101B
:100170007390223073500030970200009382420146
:1001800073901234732540F1730020309301000204
:10019000B7800000938000E03771DBB6130171DB9C
:1001A00033872002B7130000938303206314774A38
:1001B00093011002B7800000938000FC3771DBB61A
:1001C000130171DB33872002B713000093830324EC
:1001D0006312774893012000930000001301000090
:1001E00033872002930300006316774693013000A3
:1001F00093001000130110003387200293031000B6
:10020000631A77449301400093003000130170009B
:100210003387200293035001631E774293015000FD
:10022000930000003781FFFF338720029303000013
:100230006312774293016000B70000801301000051
:100240003387200293030000631677409301700008
:10025000B70000803781FFFF33872002930300003F
:10026000631A773E9301E001B7B0AAAA9380B0AABF
:10027000370103001301D1E733872002B7030100E0
:100280009383F3F76318773C9301F001B700030001
:100290009380D0E737B1AAAA1301B1AA338720020D
:1002A000B70301009383F3F76316773A93012002B3
:1002B000B70000FF370100FF3387200293030000DF
:1002C000631A7738930130029300F0FF1301F0FFB7
:1002D0003387200293031000631E77369301400298
:1002E0009300F0FF13011000338720029303F0FF07
:1002F0006312773693015002930010001301F0FF50
:10030000338720029303F0FF631677349301800054
:100310009300D0001301B000B38020029303F008D3
:10032000639A7032930190009300E0001301B000D3
:10033000338120029303A009631E71309301A00052
:100340009300D000B38010029303900A639470303E
:100350009301B000130200009300D0001301B0001D
:1003600033872002130307001302120093022000B8
:10037000E31452FE9303F008631E732C9301C00034
:10038000130200009300E0001301B0003387200245
:100390001300000013030700130212009302200051
:1003A000E31252FE9303A0096316732A9301D0004F
:1003B000130200009300F0001301B0003387200205
:1003C00013000000130000001303070013021200C3
:1003D00093022000E31052FE9303500A631C73261D
:1003E0009301E000130200009300D0001301B0005D
:1003F000338720021302120093022000E31652FEFC
:100400009303F008631877249301F00013020000AF
:100410009300E0001301B0001300000033872002B6
:100420001302120093022000E31452FE9303A0096A
:100430006312772293010001130200009300F00081
:100440001301B000130000001300000033872002E6
:100450001302120093022000E31252FE9303500A8B
:10046000631A771E93011001130200009300D0005D
:10047000130000001301B0003387200213021200A2
:1004800093022000E31452FE9303F0086314771CD8
:1004900093012001130200009300E000130000000C
:1004A0001301B00013000000338720021302120072
:1004B00093022000E31252FE9303A009631C7718F5
:1004C00093013001130200009300F00013000000BC
:1004D000130000001301B000338720021302120042
:1004E00093022000E31252FE9303500A631477161E
:1004F00093014001130200001301B0009300D000EB
:10050000338720021302120093022000E31652FEEA
:100510009303F00863107714930150011302000055
:100520001301B0009300E0001300000033872002A5
:100530001302120093022000E31452FE9303A00959
:10054000631A771093016001130200001301B000D9
:100550009300F00013000000130000003387200216
:100560001302120093022000E31252FE9303500A7A
:100570006312770E93017001130200001301B000A3
:10058000130000009300D0003387200213021200F2
:1005900093022000E31452FE9303F008631C770AD1
:1005A00093018001130200001301B000130000004A
:1005B0009300E000130000003387200213021200B2
:1005C00093022000E31252FE9303A00963147708FC
:1005D00093019001130200001301B000130000000A
:1005E000130000009300F000338720021302120072
:1005F00093022000E31252FE9303500A631C770417
:100600009301A0019300F001330110029303000055
:10061000631271049301B001930000023381000260
:1006200093030000631871029301C001B30000023C
:1006300093030000639070029301D00193001002B5
:100640001301200233802002930300006314700022
:10065000631030020F00F00F6380010093911100CE
:1006600093E111009308D005138501007300000089
:100670000F00F00F930110009308D0051305000040
:1006800073000000731000C00000000000000000B4
:10069000000000000000000000000000000000005A
:1006A000000000000000000000000000000000004A
:0C06B0000000000000000000000000003E
:1010000000000000000000000000000000000000E0
:1010100000000000000000000000000000000000D0
:1010200000000000000000000000000000000000C0
:1010300000000000000000000000000000000000B0
:081040000000000000000000A8
:040000058000000077
:00000001FF
